:020000040000FA
:100000002500290A6A002900FF0CE9010307EA011B
:100010000307250A030C2800DF0C1009040A6800F6
:100020002700E70CE7016802FC0C03071B0AE70145
:100030000306170AE7010400E803170A0706200A67
:100040002707240A0000240A0008C404A4040400AA
:1000500000086400FF0C32003600170C35000C0C51
:1000600036000600110C2600FA0C020904004606B0
:100070003A0A360A000C6606010C3B000400000C2C
:100080009B004307460A220C2600480A110C260052
:0A009000040046074C0A480A360A2D
:021FFE00EE0FE4
:00000001FF
